:1080000080DD800A0A5052494E540D0A80140A50ED
:1080100052494E540D0A801E205052494E5420227F
:10802000544154544C4554414C45204D4F44454CCB
:108030002023223B0D208028105052494E54204DC1
:108040004F44454C0D1080320A5052494E540D0A8F
:10805000803C225052494E5420222020532F4E2043
:10806000222C20534E2531303030303030303030FB
:108070000D2280462A5052494E542022284329205E
:1080800031393839204F4E53455420434F4D5055C8
:1080900054455220434F52502E220D2A80500A50F0
:1080A00052494E540D0A805A2F5052494E542022A4
:1080B0005454424153494320222C564552532F31A8
:1080C00030302C222E222C2330322C564552532570
:0D80D0003130300D2F8064084E45570D08EB
:10C000008E00FFBDF8158621BDFB1DBDC0BF42C01F
:10C010001E43C02744C03046C07253C0A100BDFBC0
:10C020001D717F147EFB4DBDFB1DBDF8157EC71C29
:10C03000BDC0DA3CBDFD21BDFB42383CC610A600A8
:10C04000BDFD26BDFB46085A26F4BDFB4238C6108E
:10C05000A60081202C02862E817F2F02862EBDFB1A
:10C060001D085A26EBBDF815BDC11F812E26C47EC2
:10C07000C000BDFB1DBDFB46BDC0ED183C862CBD00
:10C08000FB1DBDC0EDDD56862CBDFB1DBDC0ED37D3
:10C09000BDF8153238A700089C5626F9A7007EC0C7
:10C0A00000BDC0DABDFD21BDFB42A6009753BDFD1A
:10C0B00026BDFB42BDC0EDE700BDF8150820E53800
:10C0C0003CBDC11FA10027096D0027F30808082007
:10C0D000F3333336EC0118326E00BDFB1DBDFB4659
:10C0E0007F00527F0053BDC0ED187EF815BDC11F03
:10C0F000812E26037EC000810D2603DC523980305C
:10C1000025EB810A2508800725E3811024DF974667
:10C11000BDFD2EDC5205050505DB46DD5220CE7E39
:02C12000FAE043
:10C40000544154544C4554414C45204D4F44454CA7
:10C41000203520202843292031393839204F4E53E8
:10C42000455420434F4D505554455220434F525090
:10C430002E0D4C495354CB43545952554ECAE250D9
:10C4400052452A52554ECADB462452454D494E4468
:10C45000CFC0465245DD21414F4E454F4ED82F416A
:10C460004141454F4646D82A4242535441545553C0
:10C47000DD3C4E455854C960544F4C4554CEA656E9
:10C4800041524946CDEA4E4F5445474F544FCB2B6E
:10C49000454E474F535542CD955352455455524EF4
:10C4A000CDBE464F52C8D84745544255525354CE3C
:10C4B000B65853544F5245CEFC4150534554D3BB0C
:10C4C000564150434C52D445544553444FDB0331FD
:10C4D000313143414C4CDC2E3232434F554E54DE09
:10C4E0006945534C454550D33D525550524F47DB5B
:10C4F000C65855474554D54F4446544F4E45D7A787
:10C5000052535553454E44D4C62F4F4E455252D6E2
:10C51000A32352415445DE42545941534DE0B34A9E
:10C520004E4B52454DCDDB41524B5052494E54CCAF
:10C530007453584D4954D857574F53544F50CAD538
:10C54000544F4954455854D6C34F4F54455854D767
:10C550005F475354494D45D874405254494D45D9CD
:10C56000CA4041444C4F4F50DFCF494E505554CEF6
:10C570000F38585348414B45D83A4F46464C44D162
:10C5800079454F4E4C4F4144DEA744494DDCA752FC
:10C5900045414E4557CAC14F4C44434F4EDE1C44A3
:10C5A0004545CEA0544FC8FB46524F4DF4FA535464
:10C5B0004550C9104154C9164348414EE775545976
:10C5C000474554E7A326474F50494EE82154484574
:10C5D000534449EB94202020504552494F44EC7B72
:10C5E000414253E760424545535152E8BF474154E9
:10C5F00054454D50E959484953494EEA1D4F464666
:10C600004153494EEA894E55434F554E54EBE74549
:10C610004C4F47ED33494E47455850EEEE49524591
:10C6200056455253EB7D5A59534EEB8950495A4562
:10C630004D4F44454CEB7453E72C3DE5B2252F2F6D
:10C640002A343E3DE5832F233C2F3E3CE58E7E2F52
:10C650002A3C3C3EE58E2B3D2D3E3EE5A0454E441A
:10C660002E2E3C3DE5A93F2F3E3E3CE5B93C3E3CED
:10C670000404E5C00ECE71786F00088C718E26F828
:10C680001A1ABDFA7E861A97111ABDFA7E7F006AC1
:10C690007F00767F008C7F00B37F00B47F00817FB6
:10C6A0000093BCF81539BDC6747ECADECE0142DFE8
:10C6B000B1FF718ECC0400FD7070CC3FFFFD717432
:10C6C000CC5FFFFD7176CC0400FD70707F00B57FFC
:10C6D000006A7F0076860AB776E0CC1770DDAF86F9
:10C6E00039979F97A597A897A2867E97ABCCFB1DFD
:10C6F000DDACCE0142DFB1FF718ECC0000DD9ADDF2
:10C700009C7F007786FF978C979E7F00927F00B674
:10C71000BDC6747F00937EC8694F4B0DCE01429C0D
:10C72000B1270BDFB1FF718ECC3FFFFD71748E7F9F
:10C73000FF86FF979E860AB776E07F00817F008C98
:10C74000BDF815CEC7194FBDF696CEC751FF71780B
:10C75000CE0000FF7180FF717A863EBDFB1D4FCE7B
:10C7600071BCBDF5A8083CCE71BC865CBDEFF4265B
:10C770001EBDE4FEFC700093522607FC7002935429
:10C7800027033820D4865CBDEFF427037EF4FA1823
:10C7900038DF5618BDF079DC56DD4EBDF004DC52B2
:10C7A0002634DC54261B8627BDEFF427AC7EC88ACE
:10C7B00045444954494E472044495341424C45441D
:10C7C0000D7D0092270DCEC7B04FBDF696BDF81572
:10C7D0007EC7594D2A06CC00087EF1180909098A3E
:10C7E00080ED00DF46DC4E9346E702DE4E09E700AF
:10C7F000FE718E09FC718EE000820018EC00847FCF
:10C800009354FE718E2505BDF6152705FF719A20FC
:10C810001BFF7192FF719AFC718EFD7194BDF63809
:10C82000FF7190BDF787FC7192FD718EDC4E9346CF
:10C83000C10526037EC759FE718EFF7196F371966E
:10C84000FD719818BC71741823037EF59FFD718EDD
:10C85000BDF7A0FC719AFD7192DC4EFD7194DC462F
:10C86000FD7190BDF7877EC759CE8002DFB1FE8093
:10C8700000FF718ECE0142FF7174FE80008CFFFFBD
:10C8800026037EC71C7ECADE0000CCC888FD7178F6
:10C89000CCC432DD520908A600B1C41C27F8DF461B
:10C8A000A6003CDE52E6002B2811270B18C3000817
:10C8B00018DF5220F0DE4A08E600DF4A38083CE183
:10C8C0000027F2C180240838DE463CDE5220DDDE3F
:10C8D0004A08A60038363739BDF7E0BDF4B2DC525D
:10C8E000FD7180B6C41D814F2709FC71808300044F
:10C8F000FD7180CCC5A4DD527EC895BDE4FEDC543C
:10C90000FD7184DC52FD7182CCC5AEDD527EC895CE
:10C91000BDE4FE7EC91FCC0001DD545F4FDD52DC5B
:10C9200052FD7186DC54FD7188FC7178FD718AFFBF
:10C93000718C30200518C3000E18EC00271C18BCA1
:10C9400071801826F0FF719618C3000EFD719830A3
:10C95000FF719ABDF7A0FE719835FE718C7EF00BC9
:10C96000BDF01124037EF4FAFD717C3CFE7180263B
:10C9700004387EF4FABC717C270738BDF7B97EC94C
:10C980006BEC02F37188ED02EC00F97187B97186E6
:10C99000295BED00FC71862B267D71822A066D00D5
:10C9A0002A4D20046D002B39EC0018BC7182253112
:10C9B000263D18EC0218BC71842526272420307DE2
:10C9C00071822B066D002B2720046D002A13EC00CA
:10C9D00018BC71822519260918EC0218BC7184252F
:10C9E0000E38FC718AFD7178FE718C2006ED0038DE
:10C9F000BDF7B97EF00BBDE4FEDC522605DC544DDC
:10CA00002A09CC00087EF1187EF4FA3637862CBD50
:10CA1000EFF426F4BDE4FEDC5226E7DC544D2BE2B5
:10CA20003332DD48DC54934825D83CFE7178EC0065
:10CA3000847FDD502733189C48252E9C54270224E0
:10CA400028BDF815CECA4F4FBDF696387EC71C4399
:10CA5000414E4E4F5420455241534520435552526A
:10CA6000454E54204C494E450DDE54DF52DE48DF22
:10CA700054CE0142BDF6262404387EF00BFF71929D
:10CA8000DC52C30001DD54BDF6262408FC7192FD82
:10CA9000718E2012FF7190FE718EFF7194BDF78729
:10CAA000FE7192FF718EDE5027CFDF54CE0142BD62
:10CAB000F626080808A600810D27BF813A27BB206B
:10CAC000F3BDF004810D2707813A27037EC9F6CC18
:10CAD0000142FD718EBDF4EF7EC71CBDF4EF86FFF1
:10CAE0002004BDF4EF4F978C7F0081DEB17F0054AE
:10CAF0007F0055BDF62624037EC71CFF717896B5CE
:10CB0000271BBDFB1DEC00847FDD547F00527F009E
:10CB10005386019745BDF6D1863EBDFB1D0808082A
:10CB2000BDF826CCC472DD527EC895BDE4FE3CBD86
:10CB3000F4EFBDF64B270738CC00157EF1183232E2
:10CB40007ECAFBBDF01124037ECBE03CFD7196183C
:10CB5000EC00DD64EC02DD66CCF1E2DDAC387F0098
:10CB6000547F0055862CBDEFF4260DBDF079DC52C4
:10CB70002706CC00087EF118DC542BF63637964495
:10CB80002729862CBDEFF4270A862DB1C41FBDEFDF
:10CB9000F42613BDF07996442711DC5226D4DC54D8
:10CBA0002BD0DD5E200ACC00002003CC7FFFDD5EB1
:10CBB0003332DD543CBDF6152512BDF762BDF626B5
:10CBC000250AEC00847F935E27F025EEFE7196DC4B
:10CBD00064ED00DC66ED02CCFB1DDDAC387EC71CCD
:10CBE000BDF079DC522706CC00087EF118DC542B0E
:10CBF000F6363796442729862CBDEFF4270A862D72
:10CC0000B1C41FBDEFF42613BDF07996442711DCA3
:10CC10005226D4DC542BD0DD5E200ACC0000200349
:10CC2000CC7FFFDD5E3332DD549676368601977613
:10CC30003CBDF6152517BDF7627D0093262ABDF68B
:10CC400026250AEC00847F935E27EB25E9383284A1
:10CC5000019776863BBDEFF4260BBDFAE0811327E2
:10CC6000F9811127F57EC71C383284019776BDFA09
:10CC70007E7EC71C863BBDEFF426037EF00B860D3F
:10CC8000BDEFF4270C863ABDEFF427058D0A7EF040
:10CC90000B09BDF8157EF00B86019745BDF6AA2756
:10CCA000698623BDEFF42639C600A600813026022E
:10CCB000C680D745BDE4FE9655847F9A4597458644
:10CCC00048C610A10027138642C602A100270B8682
:10CCD00051C608A1002703C60A0908F776E07ECDF1
:10CCE0000AA600815C260A08BDE4FE96559DAB208D
:10CCF00019867BBDEFF4260CBDCD2F867DBDEFF4EC
:10CD000026252006BDE4FEBDF6D1862CBDEFF42716
:10CD10008B863BBDEFF4260139860DBDEFF4270A63
:10CD2000863ABDEFF427037EF4FABDF8150939BD44
:10CD3000E4FEBDCF9BDC523637DC543637862CBD43
:10CD4000EFF426E3BDE4FEBDCF9B3332DD48333242
:10CD5000DD469352250E2706CC00167EF118DC54D2
:10CD6000934825F4BDCD7EBDF221BDCD7E9DABDCCB
:10CD700046935225EF2606DC54934824E7393CDEDF
:10CD8000463CDE483CDE64DF46DE66DF4838DF6670
:10CD900038DF643839BDF7E0BDE4FEBDF4EF3CBDDB
:10CDA000F64B270738CC00157EF11818FE71783C39
:10CDB000FE717A3C7F7180BF717A187ECAFBBDF428
:10CDC000EFFC717A26037EF4FABE717A38FF717A2D
:10CDD00038FF717838BDF7B97EF00BFE71787F00AF
:10CDE000547F0055BDF6387ECAF6BDE4FEDC5226FF
:10CDF00004DC5427037ECB20BDF64225037ECAFB0C
:10CE00007EC71CBE717E38FF71783838BDF8153C7E
:10CE1000BDF6AA2609BDF011DD54256820233CBDCE
:10CE2000F011DD5424037EF4FAA600B1C41E974528
:10CE30004FA70038BDF696964509A700863ABDFB78
:10CE40001D3CFE71783CCEFFFFFF7178BF717EDC28
:10CE5000543736863ACE74BDBDF5A8CE74BDA60053
:10CE6000810D2606A7018630A700BDE4FEBDF004B3
:10CE7000810D268F380FDC54ED02DC52ED000E38A8
:10CE8000FF71783832B1C42232863BBDEFF42703FC
:10CE9000BDF815862CBDEFF426037ECE0F7EF00B79
:10CEA000A600810D270ABDF4B2862CBDEFF427F64B
:10CEB0007EF00B7EF4FABDCF82862CBDEFF426F314
:10CEC000BDE4FE3CDE522609DE5427058C000C250D
:10CED0000738CC000B7EF118183837C601D75286B8
:10CEE0002CBDEFF4260DA600803025C7810324C396
:10CEF000975208323CD652BDF92B202CBDCF8286EA
:10CF0000319762862CBDEFF4261D8623BDEFF426F3
:10CF100031A600088132270B81342707813127038E
:10CF20007EF4FA976220DC3CFE7196B6C41E814EF8
:10CF30002704DC422002DC66ED02DC64ED00387E72
:10CF4000F00BBDF0048127270481222610CCF1E2EA
:10CF5000DDACBDCC98CCFB1DDDAC7ECF27BDE4FEA7
:10CF6000D662C134260C9652BDF1E29653BDF1E271
:10CF70002004C13226059654BDF1E29655BDF1E27A
:10CF80002081BDF0112511FD71963CFE7196EC00DB
:10CF9000DD64EC02DD6638397EF4FAFC7176B3713B
:10CFA00074D39CDD48DC9AC90089009352250B2676
:10CFB00008DC4893542503270139CC00167EF1186C
:10CFC0003CFC718E8301422604387EF00B188C3FA6
:10CFD000FF2522CECFDD4FBDF6967EC71C50524FA7
:10CFE0004752414D20544F4F2042494720464F520F
:10CFF00020524F4D0018C38002FD0140CED3104F88
:10D00000BDF696BDF815CE177096431A914327FBCF
:10D01000BDFAA6260D0926F1CED3204FBDF6967E89
:10D02000C71CBDFAE0811826037EC71C811526D9CE
:10D03000CE7713DF5286019755FC718EDD4ACC7E88
:10D04000C0DD4CCE0140BDD08338862BBDEFF43C13
:10D05000260C4F5FDD4CDD4ACEC000BDD0834FCEE5
:10D06000D06EA60081242714BDD1050820F43A30E3
:10D070003030303030303030300D0A24BDD15638A9
:10D080007EF00BDF4E7F00467C0046089C4A270658
:10D090009646811026F2863ABDD1057F0047964616
:10D0A000BDD0E4DC4ED34C37BDD0E432BDD0E44F2C
:10D0B000BDD0E4DE4EA600BDD0E4089C4A27107A1D
:10D0C000004626F14F9047BDD0E4BDD0D920B44FE3
:10D0D0009047BDD0E4BDD0D939860DBDD105860AB3
:10D0E000BDD10539369B47DD47323644444444BD03
:10D0F000D0F732BDD0F739840F8B30813A25028BBF
:10D1000007BDD105393CDE52A7008C77922706086F
:10D11000DF5238393CCE7713DF524F97548601BD2A
:10D12000FB1D9655BDFB1D43BDFB1DA600BDFB1D94
:10D130009B549754088C779326F19654BDFB1DBDE4
:10D14000FAE0811527CF81062707811826C77EC7F9
:10D150001C7C00553839DE528C7793270B6F000802
:10D160008C779326F8BDD1148604BDFB1DBDFAE073
:10D17000811827DA810626DE39BDE4FEBDCF9BDCAF
:10D1800052DD64DC54DD66862CBDEFF427037EF4AB
:10D19000FABDE4FEBDCF9BBDD3052406CC00167EB0
:10D1A000F118B6C41F81532708DC529A40DA41DDDA
:10D1B0005218DE523CDE543C18862CBDEFF4270793
:10D1C000CC177036372020BDE4FEDC522706CC0099
:10D1D000177EF118DC543637862CBDEFF42608BDD7
:10D1E000F01124067EF4FACC004EDD4E3332DD50D1
:10D1F0001838DF5438DF52183CDE4E8C004E260AB9
:10D20000CED3104FBDF696BDF815BDD2232626DE2F
:10D210004E8C004E260ACED3204FBDF696BDF81593
:10D220007ED2F7DE5096431A914327FBBDFAA6261D
:10D23000030926F139BDFAE0811826037ED2F78171
:10D240001526C78601974720347C0047BDD2232688
:10D250000D3338BDD30524037ED2D77ED2F7BDFA75
:10D26000E0333881062716811826037ED2F7811510
:10D2700027043C3720D6DF66D7657A0047BDD30543
:10D28000254BDE663CD665377F005A7F005B860102
:10D29000BDFB1D9647BDFB1D43BDFB1DBDD3052535
:10D2A00015965A8180271EBDF221BDFB1D9B5B9701
:10D2B0005B7C005A20E6965A818027094FBDFB1DF2
:10D2C0007C005A20F1965BBDFB1D7ED2498604BDD1
:10D2D000FB1DBDD2232619730064730065DC664311
:10D2E00053C30001DD66DC64C9008900DD642007EA
:10D2F000BDFAE0810626D6DE4EDC64ED00DC66ED8C
:10D3000002387EF00B965390652604DC5493663900
:10D3100057414954494E4720464F52204E414B00F9
:10D320004E414B204E4F5420464F554E44204245CF
:10D33000464F52452054494D454F555400BDE4FEDB
:10D34000DC522706CC00187EF118DC54260D9643DB
:10D350001A914327FB4FDD6C7EF00BDD6E20010838
:10D36000A600B1C42227F8813A272C810D27283C3A
:10D3700020091ADC6C936E270B24097B401527F2D9
:10D38000387ECB20DD6C38CC0000DD54BDF6422564
:10D39000037ECAFB7EC71C3C1ADC6E936C270925F2
:10D3A000022AF5862ABDFB1DCE0000DF6C387EF018
:10D3B0000B9DA53838CC000C7EF118BDE4FEDC5284
:10D3C000270DCC000C7EF1183C8DE6387EF00BDC8E
:10D3D000544D26F4C11124F0C108241786805D271E
:10D3E00004445A20F9369A159715329A8B9720974C
:10D3F0008B203EC10E2421C00886805D2704445A3C
:10D4000020F9B1C42224024444369A039703329A85
:10D410008A9701978A7ED431C00E86015D27044821
:10D420005A20F9369A179717329A709716977020E4
:10D4300000862CBDEFF427837EF00B9DA83838CCF6
:10D44000000C7EF118BDE4FEDC52270DCC000C7EF2
:10D45000F1183C8DE6387EF00BDC544D26F4C111FA
:10D4600024F0C108241886805D2704445A20F93628
:10D470004394159715329A8B9720978B203EC10EB7
:10D480002422C00886805D2704445A20F9B1C422B2
:10D4900024024444364394039703329A8A970197AF
:10D4A0008A7ED4BCC00E86015D2704485A20F93616
:10D4B0004394179717329A7097169770862CBDEF82
:10D4C000F427827EF00BBDD63586809A8A97019725
:10D4D0008ABDF0048122270481272610CCD522DDC5
:10D4E000ACBDCC98CCFB1DDDAC7EF00BBDD67DDC9D
:10D4F0007B2604DC79271BBDF221BDD522DC7B8392
:10D500000001DD7BDC79C2008200DD7926E9DC7B6D
:10D5100026E53CFE7196DC64ED00DC66ED02387EAB
:10D52000F00B3CDE7D8C011324010FBDD62F717FE3
:10D5300003BDD62FC608442505717F0320057280E0
:10D54000032000BDD62F5A26ED728003380E39BD58
:10D55000D635BDD67D862CBDEFF427037EF4FABD0B
:10D56000E4FEDC7B2607DC7926037ED51286FE945A
:10D570008B9720978B867EB7010CCCD5E0FD010DF3
:10D58000DC522706CC00257EF1180FDC42D354DD97
:10D5900054DC40D9539952DD5296AE8900974E7FA4
:10D5A000007FDF467F0080DC7D83011325037A0046
:10D5B000800E01010F7201140E1A0F967F26169627
:10D5C0004E90AE251026EADC529340250826E2DC78
:10D5D00054934224DC71FE140E86FF97807ED51290
:10D5E00071FE14968027010EDC7D04D37D18BDD614
:10D5F00031C68096150425070101BDD62F20F417EA
:10D60000DE46BDF1E2DC7B830001DD7BDC79C2001C
:10D610008200DD79DC7D04047B0115260583000191
:10D6200026F6DC792608DC7B260486FF977F3BDE26
:10D630007D0926FD39BDE4FE3CDC52DD46DC54DDCF
:10D6400048BDF197CC04B07B01BB2703CC0960DD5A
:10D6500053BDF2BADC52260CDE548C0FA024058C8C
:10D66000001E240A38CC00197EF1187EF4FA1883C3
:10D670000007DD7D38862CBDEFF426EF39BDE4FED2
:10D68000DC52DD79DC54DD7B862CBDEFF426DCBD7D
:10D69000F01125D7FD71963C18EC00DD64EC02DD3D
:10D6A000663839BDE4FEBDF4EF3CBDF64B270A38C1
:10D6B0007F0081CC00157EF118DF823886FF9781CC
:10D6C0007EF00BBDCF82860DB77198862CBDEFF42E
:10D6D0002616865CBDEFF42636BDE4FE9655B7717E
:10D6E00098862CBDEFF427273C4FCE74BDF6719879
:10D6F000BDF5AACE74BDA600B17198270C08DF5203
:10D7000038BDF1E23CDE5220EDBDF1E27ECF28BD16
:10D71000E4FEDC522706CC001A7EF118DC542732D6
:10D72000DC54DD52BDFAA6270FBDFAE036BDF1E2AA
:10D7300032B17198271920E896431A36BDFAA632FD
:10D7400026E7914327F4DC52830001DD5226E97E6F
:10D75000CF27BDFAA627F8BDFAE0BDF1E220F0BD63
:10D76000CF82860DB77198862CBDEFF42612865CA9
:10D77000BDEFF427037EF4FABDE4FE9655B7719829
:10D780003CBDF221B171982705BDF81720F338365A
:10D79000863BBDEFF432270C810D2605BDF8152020
:10D7A00003BDFB1D7ECF27BDE4FEDC522706CC0067
:10D7B0001B7EF118DC54188C006E1825F136378664
:10D7C0002CBDEFF426E8BDE4FEDC5226E1DC542655
:10D7D000043232203505DD5425D43332DD463C8613
:10D7E0007EB70106CCD80DFD010771FD039608DC5C
:10D7F00009D346DD0B8601970F860897081ADC4689
:10D8000026FB7F00088600970F387EF00B9608DE17
:10D8100054270E09DF5488019708DC0BD346DD0B33
:10D820003BDC0BD346DD0BDF463B86FF3620024F49
:10D8300036BDF4EF3297927EC71CBDE4FEDC522762
:10D8400006CC001C7EF118DC542706DDAF860120D3
:10D85000014F97767EF00BA600812D260DBDFAAB09
:10D8600026FB86FF0897777EF00B812B27037EF43B
:10D87000FA4F20F0B6719CBA719DBA71A0BA71A12D
:10D88000BA71A4BA71A5BA71A8BA71A9BA71AAF687
:10D8900071AB271FC12025028AFFBA71ACBA71ADE6
:10D8A000BA71AEF671AF270BBA71B0BA71B1BA7175
:10D8B000AA2706CC00267EF1187F004A7F004BFC89
:10D8C000719EDD4CCC003CDD484F5FDD46DD52FCF7
:10D8D00071A2DD54BDF3EEBDD9AF4F5FDD46DD5221
:10D8E000CC0E10DD54FC71A6DD48BDF3EEBDD9AF02
:10D8F0004F5FDD465CDD52F671AB5ADD48CC51809E
:10D90000DD54F671B3C1292404CB142008C050257E
:10D9100015C1142411D75E54545C4FD348DD48F62A
:10D9200071AFC10D2506CC001D7EF118D7463CCE47
:10D93000D9BEC1032409D65EC40326037A00495F19
:10D940007A00462707EB0089000820F438D348DD29
:10D9500048BDF3EEBDD9AF4F5FDD52D65EDD54CC8E
:10D9600001E1DD46CC3380DD48BDF3EEBDD9AFBD6E
:10D97000F011250E3C18DC4AED00DC4CED02387E3F
:10D98000F00BDC4CDD484FD64BDD465FDD52C66404
:10D99000DD54BDF3EE0FDC50DD42D64FD741866437
:10D9A000D64A3DDB4E8900D74097AE0E7EF00BDCA9
:10D9B00050D34CDD4CDC4ED94B994ADD4A391F1C03
:10D9C0001F1E1F1E1F1F1E1F1E1FBDF0113C2446C1
:10D9D0000F96AE9752DC40DD53DC4297550ED75E72
:10D9E000CC0064DD485FDD46BDF2BADC53DD5F96F6
:10D9F0005597619651D65EDD544F5FDD52DD46C6C8
:10DA000064DD48BDF2BADC549B61DD54DC5FC900C3
:10DA10008900DD52200918EC02DD54EC00DD5218BB
:10DA20008C8000250738CC001E7EF118CC0001DD6B
:10DA300046CC5180DD48BDF2BADE543CDC4EDD52AE
:10DA4000DC50DD544F5FDD46CC0E10DD48BDF2BA30
:10DA5000DC54FD71A65FFD71A4DC4EDD52DC50DDAF
:10DA6000544F5FDD46CC003CDD48BDF2BADC54FDCE
:10DA700071A25FFD71A0DC50FD719E5FFD719C384D
:10DA8000187F00527A00527C0052BDDAF3260A83D6
:10DA9000016E24F3C3016E200883016D24E9C301E4
:10DAA0006D3637D652CB50C1642502C0644FFD712C
:10DAB000B25FFD71B03332CED9BE7F00547F0053C8
:10DAC0007C005337E600BDDAF3260937D653C1028E
:10DAD0003326015C08D75533935424E4D3544F5C68
:10DAE000FD71AAD653FD71AE5FFD71A8FD71AC3812
:10DAF0007EF00B36965284033239CC00207EF1182A
:10DB00007EF4FABDF0048122270481272613BDDBB1
:10DB1000B2CCDB95DDACBDCC98CCFB1DDDAC7EF092
:10DB20000BBDE4FE18DE523CDE543C18862CBDEFE3
:10DB3000F426CDBDE4FEDC5226C0965426BCD65554
:10DB40002750C12124B4BDDBB2D7461838DF543882
:10DB5000DF5218D64686209046270F780055790068
:10DB6000547900537900524A20EF7B805227057286
:10DB70000403200371FB0372041571FB1578005533
:10DB80007900547900537900525A26DE72201571BB
:10DB9000DF157EF00BC608492405720403200371CB
:10DBA000FB0372041571FB155A26EC72201571DF08
:10DBB000153986049A8A9701978A86249A8B97202A
:10DBC000978B71DB15398627BDEFF4270A8622BDB6
:10DBD000EFF427037EF4FABDDC02974EBDDC02367B
:10DBE000BDDC021632DD46BDDC02BDDC02D64E27AE
:10DBF0000E5AD74E3CDE46A70008DF463820EB7EA3
:10DC0000F00B8D0A48484848368D03331B39A6006F
:10DC1000088030250C810A250B80072504811025FA
:10DC2000037EF4FA39CC00217EF1187EF4FABDE4CB
:10DC3000FEDC5226F0DC54183C18862CBDEFF4268E
:10DC4000EABDF0048122270481272610183818DD48
:10DC5000ACBDCC98CCFB1DDDAC7EF00BBDE4FE185A
:10DC6000DE523CDE543C18862CBDEFF42705CC0078
:10DC70004E2005BDF01125B3FD71961838DF5438DC
:10DC8000DF5238DF46183CBDFAAB26FBCEDC983CB1
:10DC9000DE463CDC54DE52393CFE7196ED0218380B
:10DCA00018ED00387EF00B8628BDEFF42664BDE445
:10DCB000FEDC522666DC54363705255F052556DD29
:10DCC00054CC6FFF935425533637862CBDEFF42682
:10DCD00041BDE4FEDC5226433332DD463CCE0142F8
:10DCE0009CB138270BFD7176CC0142FD7174201375
:10DCF0009354252118BC718E18251AFD7174DC46C9
:10DD0000FD71763332FD70708629BDEFF426037EF7
:10DD1000F00B7EF4FACC00227EF118CC00237EF1C9
:10DD200018BDF4EFFC7174B3718EDD547F00527F27
:10DD3000005386069745BDF6D17EC71CBDF4EF3C67
:10DD4000CEDDCD4FBDF6967F00527F00537F00455C
:10DD5000FC718E830142DD54BDF6D1CEDDDE4FBDB8
:10DD6000F696FC7174830142DD547F00527F0053AC
:10DD70007F0045BDF6D1BDF815CEDDE24FBDF6966C
:10DD80007F00527F00537F0045FC7070DD54BDF66C
:10DD9000D1BDF815CEDDF84FBDF696FC7176B371A6
:10DDA00074D39CDD54DC9AC9008900DD527F0045A4
:10DDB000BDF6D1CEDE0F4FBDF696FC7174C30001E7
:10DDC00018BDFD218648BDFB1D38BDF00B2020206D
:10DDD0002020202050524F4752414D3A2000202F02
:10DDE0002000202020202020204020415252415954
:10DDF0002053495A453A200020202020202020444A
:10DE000041544146494C452053495A453A20002C3B
:10DE10002053544152545320415420007F00B37F7B
:10DE200000B4867BBDEFF4260EBDF011250CDDB3EA
:10DE3000867DBDEFF426037EF00B7EF4FAC6317EBC
:10DE4000F118BDE4FEDC5226F4DC5427F04D26ED3B
:10DE5000D7B786C05F5C90B724FB5A7B01BB260115
:10DE6000545AD71CD7637EF00B7F0008BDF01125F4
:10DE70001CFD76DE867EB70109CCDE90FD010AC668
:10DE800002D708D608DC0DDC09C612D7087EF00BD5
:10DE90009608FE76DEEC02C30001ED02EC00C9003C
:10DEA0008900ED00DE0D3B86FF974F860197503CC1
:10DEB000CC0052FD7198BDF01125123637862CBD6D
:10DEC000EFF426073332FD71982002323338BDE477
:10DED000FEDC52DD64DC54DD66862CBDEFF42703E6
:10DEE0007EF4FABDF01125F8FD71963C96B63686A3
:10DEF0001897B6BDFA7ECE006496431A914327F96F
:10DF0000BDFAA626EE0926F18615BDFB1D7C004F45
:10DF1000D64FC11426208618BDFB1DFE71964FED0D
:10DF2000025FED00FE7198DC66ED02DC64ED00320C
:10DF300097B6387EF00BBDDFBB27CDBDFAE0811868
:10DF40002604C61520D5810426098606BDFB1DD6EC
:10DF50004F20C88101269CBDDF6626978606BDFB43
:10DF60001D7C005020D0CE74BDC683BDDFABA700A2
:10DF7000085A26F7FC74BD5311270139CE74BF4FE0
:10DF8000AB00088C753F26F8B1753F270139B67490
:10DF9000BD4C915026064A9150270139CE74BFA638
:10DFA00000BDF1E2088C753F26F5393CBDDFBB387A
:10DFB0002704BDFAE03938387EDEF3CE01F4BDFA2D
:10DFC000A627013996431A914327F90926F0393CCF
:10DFD000BDF895961784CF971784BF971786FFB71C
:10DFE0006F835FBDE0765F1A0FCEE004FF01100E75
:10DFF000387EF00B30CC0032A702E701CCF118EDEF
:10E00000057EE06EB66F8326037EE068F66F77BD0F
:10E01000E076FA6F67FD6F7EFC7174F36F7A180813
:10E02000BC717624CFFC6F7EED00FE6F7A0808BCD1
:10E030006F6E2503FE6F72FF6F7ADE6C08DF6C7AFD
:10E0400000B82619DC42C30001DD42DC40C900896A
:10E0500000DD4096AE890097AE96B797B8717F1BEA
:10E06000FE6F6A27026E003B724017BDF89CCEFC23
:10E0700036FF011020C472401771BF17175F484860
:10E080004848CE000A71EF170524057220172003B7
:10E0900071DF177210177B08172702CB400926E59E
:10E0A00036961784EF9D28323938CC00017EF1185E
:10E0B0007EF4FABDF011240ABDF079964427F1CC24
:10E0C0000052FD71963C18EC0026DEEC02FD7198C2
:10E0D00038862CBDEFF426D87EE0EF863BBDEFF40A
:10E0E00027F63CFE7196FC7198ED02387EF00BCC61
:10E0F000E31CDD46BDF004DF483CDE46A1002609F6
:10E1000008DF463808A60020F0A6002B1908A60054
:10E110002AFB0808A6002604387EF4FADF4638DE1B
:10E1200048A6007EE0F93C16584FC3E30618EC0001
:10E13000186E0038A601BDE2FA387EE0DB38A60191
:10E14000BDE2FA38BDE4FEDC5227037EF118DC5450
:10E150002718830001B371984D2606C18024EC2056
:10E160000881FF26E6C18025E217BDE2FA7EE0DBEA
:10E1700038A60138E600C1412706C14226058B10AA
:10E180000820E736BDE4FEBDE2C1270C328B30BD6E
:10E19000E2FABDE2DB7EE0DB32BBC422BDE2FABDC7
:10E1A000E2E67EE0DB38A6013836BDE4FEDC52272D
:10E1B000037EF118DC544D26F837862CBDEFF4278A
:10E1C000037EF4FABDE4FEDC5226E6DC544D26E183
:10E1D000BDE2C12616DF46183332BDE2FA17BDE2B2
:10E1E000FA1817BDE2FADE467EE0DBDF461833326E
:10E1F0008B107EE1DA38A601387EE18338A601383B
:10E20000E600C1412709C14227037EF4FA8B40365C
:10E21000088623BDEFF4262EBDE4FE32BDE2FABD32
:10E22000E2E67EE0DB38A6013836B6C41E802BBDA0
:10E23000EFF42612BDE4FE32BDE2FABDE2DB7EE081
:10E24000DB38A6013836BDE4FEBDE2C1260C328BB8
:10E2500020BDE2FABDE2E67EE0DB9654270C328B6D
:10E2600030BDE2FABDE2DB7EE0DB328B1020E2382B
:10E27000A601BDE2FA38BDE4FEBDE2E67EE0DB3891
:10E28000388622BDEFF42604167EE2948627A1008C
:10E29000260D1608A6000811270BBDE2FA20F5BDD1
:10E2A000E4FEBDE2E6862CBDEFF427D57EE0DB3848
:10E2B00038BDE4FEBDE2DB862CBDEFF427F37EE043
:10E2C000DBA600B1C41C26030820F6812C260B080F
:10E2D000A60008815827037EF4FA39DC52260E96F0
:10E2E00054BDE2FA200EDC522706CC00277EF1183E
:10E2F000965426F99655BDE2FA393CFE7198A7006E
:10E3000008FF71983839E133E13DE170E1A5E1F5AD
:10E31000E1FCE225E241E26FE27FE2AF4E4F508046
:10E32000014C535244800441534C448005544150A5
:10E3300080065450418007494E5880084445588013
:10E3400009434C56800A534556800B434C43800C7E
:10E35000534543800D434C49800E534549800F532C
:10E360004241801043424180115441428016544240
:10E370004180175847445880184441418019534CF4
:10E3800050801A414241801B5453588030494E53AB
:10E39000803150554C41803250554C428033444579
:10E3A000538034545853803550534841803650532D
:10E3B0004842803750554C58803852545380394128
:10E3C0004258803A525449803B50534858803C4D03
:10E3D000554C803D574149803E535749803F4252FA
:10E3E00041812042524E81214248498122424C5370
:10E3F000812342434381244243538125424E458138
:10E40000264245518127425643812842565381294D
:10E4100042504C812A424D49812B424745812C4232
:10E420004C54812D424754812E424C45812F4E45FC
:10E43000478240434F4D82434C53528244524F5285
:10E440008246415352824741534C8248524F4C823C
:10E4500049444543824A494E43824C545354824D69
:10E46000434C52824F41494D83614F494D83624530
:10E47000494D836554494D836B4A4D50844E5355E5
:10E48000424486834144444486C3435058868C4C5E
:10E49000444486CC4C4453868E4C445886CE5355C7
:10E4A000428580434D5085815342438582414E448D
:10E4B000858442495485854C44418586454F528523
:10E4C0008841444385894F5241858A414444858B24
:10E4D0005354414187875354414287C7535453870C
:10E4E0008F4A5352878D53544487CD53545887CF06
:10E4F000425352888D4442890044578A0000BDE54A
:10E500002EF6C422A600081127FA817C27020939B9
:10E51000DC543736DC523736BDE52E32339A52DAC8
:10E5200053DD5232339A54DA55DD547EE501BDE5B0
:10E530005EF6C41CA600081127FA812627020939B5
:10E54000DC543736DC523736BDE55E32339452D474
:10E5500053DD5232339454D455DD547EE531BDE65B
:10E5600004A60008B1C42B27F809813C2504813F8B
:10E57000250139DC543736DC523736CCC63ADD5209
:10E580007EC895BDE5C9250B860197552008BDE5D8
:10E59000C926F57F00557F00547F00537F00523914
:10E5A000BDE5C927EE25EC20DFBDE5C927DA25D872
:10E5B00020E1BDE5C926DC20CFBDE5C924D520C8B2
:10E5C0003233DD523233DD5439DF4E381838DF5004
:10E5D00038183C183CDE503CDE4EBDE6043233DDDC
:10E5E000463233DD4896469852182A0CDE529C4635
:10E5F0002610DE549C481839DE469C522604DE481C
:10E600009C541839862DBDEFF42606BDF1977EE6A1
:10E610005D862BBDEFF4BDE66E862BBDEFF426358F
:10E62000DC543736DC523736BDE66E3233DD4632E7
:10E6300033DD48DC54D348DD54DC52974ED947993A
:10E6400046DD52964E98462BD0964E98522ACACC0A
:10E6500000097EF118862DBDEFF4270139DC54370F
:10E6600036DC523736BDE66EBDF17F7EE62BBDE768
:10E6700002862ABDEFF42621DC523637DC543637C9
:10E68000BDE7023332DD483332DD46BDF398DC4E60
:10E69000DD52DC50DD547EE671A600812F27058116
:10E6A000252701393C087F00447D00522A067C0062
:10E6B00044BDF17FDC523637DC543637964436BDE4
:10E6C000E7023297447D00522A067A0044BDF17F6A
:10E6D000DC52DD46DC54DD483332DD543332DD526A
:10E6E0003CBDF2BA38183836A60081252608DE4E21
:10E6F000DF52DE50DF54321896442703BDF17F7E8F
:10E70000E6710908A600812027F981302504813AA5
:10E7100025308128273E81262728A6018141250C06
:10E72000815B2408CCC5B8DD527EC895BDF011DDF3
:10E7300052251E3C0FDE52EC00DD52EC020EDD5481
:10E740003839BDF07996442708398628BDEFF4277B
:10E75000047EF4FA08BDE4FE8629BDEFF426F23902
:10E76000BDE74A96522A03BDF17F96522B0139CC60
:10E77000000A7EF118BDE74ADC522706CC000B7E6A
:10E78000F1183C8D0838DD545F4FDD5239DE548C72
:10E79000000B250A9D9F3838CC000B7EF11818BD60
:10E7A000F8963918FE71963CDE643CDE663C1886AD
:10E7B00028BDEFF42629BDCF827F00527F00537F12
:10E7C0000054862CBDEFF426288623BDEFF4260FD7
:10E7D000A600088134270B81322711813127127E50
:10E7E000F4FABDF2219752BDF2219753BDF2219761
:10E7F00054BDF22197553CFE7196DC66ED02DC6457
:10E80000ED00381838DF6638DF6438FF71961886F7
:10E8100029BDEFF426C9399DA23838CC000C7EF111
:10E82000188628BDEFF42670BDF197DC5405373605
:10E83000BDE4FEDC52270CCC000C7EF1183C8DD7D9
:10E8400038203ADC544D26F5C11124F1C108244C7E
:10E8500086805D2704445A20F93643948B9720978D
:10E860008B3294157EE87DC00E86015D2704485AE0
:10E8700020F9364394709716977032941727073211
:10E8800033C3000120023233DD54862CBDEFF42760
:10E890009A8629BDEFF427037EF4FA39C10E24C706
:10E8A000C00886805D2704445A20F9B1C42B240295
:10E8B00044443643948A9701978A32940320BEBD1C
:10E8C000E74A96522A06CC000D7EF118CC0000DDF6
:10E8D00046DD48DD4EDD50DD4CCC4000DD4A860F84
:10E8E000975ADC48D350DD58DC46D94F994EDD5657
:10E8F000DC58D34CDD58DC56D94B994ADD567400B0
:10E900004E76004F760050760051DC529356251E0D
:10E910002606DC5493582516DC56DD46DC58DD48C7
:10E92000DC50D34CDD50DC4ED94B994ADD4E74009F
:10E930004A76004B76004C76004D74004A76004BC8
:10E9400076004C76004D7D005A2609DC4EDD52DC07
:10E9500050DD54397A005A2089BDE74ADC52270637
:10E96000CC000E7EF1183CDC54040453D74E1658EC
:10E970004FC3E99B18EC02DD46EC0093469748969E
:10E980004E3D97499648D64E3DDB498900D346DD3A
:10E99000542A067A00527A0053383940D840D83584
:10E9A000482E8629F4268423C8217A1F7C1DC41C86
:10E9B000341AD6198C1856173E163A1540145A13A5
:10E9C0007412A211D01108104A0F960EE20E2E0DED
:10E9D000840CDA0C3A0B9A0AFA0A5A09C409240878
:10E9E0008E07EE075806C2062C058C04F604560363
:10E9F000C00320028001D6012C0082FFD8FF1AFE3E
:10EA00005CFD9EFCCCFBF0FB0AFA10F90CF7E0F67B
:10EA1000A0F524F376F15AEE80EA20EA20BDE74A19
:10EA20003C7D00522A09DC545343C38001DD54DC91
:10EA300054847FDD52188C4000182505CC8000934B
:10EA400052DD46164F05C3EAF218EC00DD48EC0231
:10EA5000A300974E96473D97517F0050D64E96475C
:10EA60003DD350D3487F00527F00537D00542A1578
:10EA70004353730052730053C3000118DC52C900A2
:10EA80008900DD5218DD543839BDE74A3C7F005615
:10EA90007D00522A06BDF17F7A0056DC52270738E6
:10EAA000CC000F7EF118DC5427462BF3CEEAF27F20
:10EAB0000057EC00189C5418240708087C005720C5
:10EAC000F1DD4A0909EC00DD4CDC4A934CDD48CE0F
:10EAD0000000DF46DC54934CDD537F0055BDF2BA95
:10EAE00096574A5FD354DD547D00562703BDF17F0E
:10EAF0003839000003240648096A0C8C0FAB12C891
:10EB000015E218F91C0B1F1A2223252828262B1F73
:10EB10002E1030FB33DE36BA398C3C563F1741CECF
:10EB2000447A471C49B44C3F4EBF5133539A55F574
:10EB300058425A825CB35ED760EB62F164E866CFFC
:10EB400068A66A6D6C236DC96F5E70E2725473B50E
:10EB500075047641776B788479897A7C7B5C7C2933
:10EB60007CE37D897E1D7E9C7F097F617FA67FD8A7
:10EB70007FF57FFFCC0005DD545FDD5239CC00E02E
:10EB8000DD547F00527F005339CC000020F2CC00CE
:10EB9000107EF118BDE74ADC5226F3965426EFD6D4
:10EBA00055BDF1975D27E7C12124E386BF948A977D
:10EBB00001978A968B8A14978B972071EB157210A8
:10EBC000152012780055790054790053790052725B
:10EBD000041571FB157B400327037C00555A26E37F
:10EBE00039CC00117EF118BDE74ADC5226F3DC5423
:10EBF00027403C18968A84FE9701978A867EB70143
:10EC000009CCEC33FD010A7F00547F005596431A6E
:10EC1000914327FB01010101D608DC0D9643C61282
:10EC20000FD7080E1A914327F796430926F27F0063
:10EC3000083839960884EF9708DC0DDC54C30001CE
:10EC4000DD54DC52C9008900DD523B9608DE4A08DB
:10EC5000DF4A84E29708DE0DDF54B4C41C270EDEC1
:10EC6000548C80002407DE5208DF52DC093B9608F2
:10EC700020F47EF4FACC00127EF1188628BDEFF461
:10EC800026F0BDE4FEDC5226ECDC5427E8183C18E4
:10EC9000862CBDEFF426DBBDE4FEDC5226D7DC5427
:10ECA00027D3DD4E183818DD508629BDEFF426C273
:10ECB0003C968A84FE9701978A867EB70109CCEC40
:10ECC0004BFD010A867EB70103CCEC6EFD01047F8B
:10ECD000004A7F004B7F004CC602D708D608DC0DE7
:10ECE000DC099643C6160FD7080E1A9143270996DA
:10ECF00043DE4E092731DF4E0FDE4A092611964CBE
:10ED0000260D7C004CDE52DF46DE54DF4820D79CC7
:10ED10005026D30E7F0008DC549348DD54DC52D2D9
:10ED2000479246DD5238397F0008CC0000DD52DDC5
:10ED3000543839BDE74A7F005ADC522A06CC00130A
:10ED40007EF1183C271574005276005376005476F5
:10ED500000557C005ADC5226ED2011DC5427DE2BB6
:10ED60000B7800557900547A005A20EF7F00467FD7
:10ED70000047DC54C3B172DD487C0047CCB172DD82
:10ED800052CC17ADDD54BDF2BADC54DD567F0058CD
:10ED9000DC4FDD52965197547F0055BDF2BADC54DA
:10EDA000D357DD57965689009756965680809756CA
:10EDB000DC5805DD58DC565949DD56730056DC57E2
:10EDC0004353C30001DD57965689009756CE000085
:10EDD000DC56DD54DD482A03CEFFFFDF52DF46BD9F
:10EDE000F398DC4EDD5EDD54CC994BDD48CC000061
:10EDF000DD46DD52BDF398DC4EC3F622DD54DC5E09
:10EE0000DD48CC0000DD52DD46BDF398DC4EC3E2A8
:10EE1000A8DD60CC0002DD5EDC57DD544FD6562AFB
:10EE20000286FFDD52DC54363705DD58DC523637BA
:10EE30005949DD56CC0000DD46974896609749BD9C
:10EE4000F398DC4FD358DD58DC56C9008900DD56F5
:10EE50004FD64E2A0286FFD356DD56D661D74933A8
:10EE600032DD523332DD54BDF398DC4ED358DD58D9
:10EE7000DC56C9008900DD564F5F7D004E2A03CC69
:10EE8000FFFFD356DD56DC5783875DDD53965682F0
:10EE90000097524F965A9B529752DC53DD543637A7
:10EEA0004FD6522A0286FF3637DD5286B19749CCBB
:10EEB0000000DD469748BDF398DC4EDD56DC50DDA2
:10EEC00058C672D7493332DD523332DD54BDF39820
:10EED000DC4ED357DD548600D6562A0286FFC90081
:10EEE00089007D004E2A03C3FFFFDD523839BDE79C
:10EEF0004ADC522B0B83000A2506CC00147EF11845
:10EF0000DC52DD56DC54DD58DC53DD549652975309
:10EF1000CC0001DD46CC62E4DD48BDF398D64E2A34
:10EF20000CC1F02408CC0000DD52DD54394F5CD711
:10EF30005A2A0286FFDD5416DD52CCB172DD487FBD
:10EF400000467F0047BDF398DC509358DD54DC4EFB
:10EF5000D2579256DD52DC524756DD5EDC5446569F
:10EF6000DD608607975B3CCCFFFFDD52CCFFF3DD15
:10EF700054CEEFD8BDEFA47A005B26F8965A2B1337
:10EF8000270F7800557900547900537900524A26AA
:10EF9000F138397700527600537600547600554C9C
:10EFA00026F13839DC5EDD46DC60DD48BDF398963D
:10EFB0005048DC4E5949DD54CC00007D004E2A03F8
:10EFC000CCFFFFDD52EC02D354DD54EC00D9539951
:10EFD00052DD5208080808390000005BFFFFFDDE23
:10EFE00000000AABFFFFD55500008000FFFF0000C6
:10EFF00000010000160908A600812027F908112742
:10F0000001093908A600812027F939BDF4D57EF41D
:10F01000FA0908A600812027F9813F262608A600C4
:10F02000812027F981282705CC00400C39BDE74A0B
:10F03000DC522627DC544D2622C106241E0505C3BA
:10F04000719C398040240139262008BDE74ADC52F2
:10F050002609DC5418BC7070182506CC00027EF11D
:10F060001805054353C370010C39811B25020D3966
:10F07000084848164FC3700039BDF1977F0044BD62
:10F08000F0047F0046812626037EF1398130240179
:10F0900039813A250139840F7D0044260A7C0044D9
:10F0A000975508A60020E57C0044D644C1052414E9
:10F0B0009747DC5405DD540505D354D346DD540889
:10F0C000A60020C89747DC5405DD54DD50DC5259BA
:10F0D000492B42DD52DD4E78005179005079004FC6
:10F0E00079004E2B3078005179005079004F79002B
:10F0F0004E2B22DC54D350DD54DC52D94F994E2B89
:10F1000014DD52DC54D346DD54DC52C90089002B97
:10F1100004DD5220AACC00033CCEF11F7EF500484E
:10F120004F573F20204552524F522023005748410D
:10F13000543F0D534F5252590D08A60081482709DC
:10F1400009399644260209093908A600803025F2BB
:10F15000810A250A8007810A25E8811024E47C00C1
:10F1600044D644C10924AEC60478005579005479C8
:10F1700000537900525A26F19B5597557EF14973F9
:10F180000052730053DC544353C30001DD54DC527E
:10F19000C9008900DD52397F00527F00537F00543F
:10F1A0007F0055393CFE71783CCEF1CCFF7178BDC3
:10F1B000F1E238FF717838393CFE71783CCEF1CC01
:10F1C000FF7178BDF22138FF7178383900010044B1
:10F1D00041544146494C45204F56455252414E47B5
:10F1E00045003CBDF1E8383936DC64260EFC71760A
:10F1F000B37174189C661827082412FC7176B371D9
:10F200007418329D943838CC00047EF118FC717467
:10F21000D366180832A70036DC66C30001DD66320B
:10F22000393CBDF2273839DC64260EFC7176B371A7
:10F2300074189C661827082411FC7176B371741831
:10F240009D973838CC00057EF118FC7174D3661890
:10F2500008A60020C25F2002C601F775D936FF75E7
:10F26000D7DC66B375D7FD75D7DC64C2008200FDBC
:10F2700075D5DC9AB375D5250B260BDC9CB375D7F9
:10F28000250226023239FC75D6050536FC75D78471
:10F290003FC3C0001833B675D92717320FBD75BDEF
:10F2A0000E36DC66C30001DD66D665C900D765325F
:10F2B0003839320FBD75C90E20E7DE46264BDE48D1
:10F2C00026083838CC00067EF118DE52263BDC5486
:10F2D000CE00007C005278004979004824F5760081
:10F2E0004876004993482404D3482001087A005204
:10F2F000270B18051874004876004920E7DF54CE24
:10F300000000DF52DF4EDD50397F004ADE52DF4E13
:10F31000DE54DF50CE0000DF52DF547C004A78001C
:10F320004979004879004779004624EF760046760F
:10F330000047760048760049DC509348DD50DC4EAB
:10F34000D2479246DD4E2410DC50D348DD50DC4ECF
:10F35000D9479946DD4E20127C0055240D7C00547F
:10F3600024087C005324037C00527A004A271A7830
:10F3700000557900547900537900527400467600A4
:10F380004776004876004920AF393CCE00468610CB
:10F390006F00084A24FA38397F00447D00522A065B
:10F3A0007C0044BDF17F7D00462A1A7A0044730038
:10F3B00046730047DC484353C30001DD48DC46C9BF
:10F3C000008900DD46BDF3EE964E2A06CC00077E8E
:10F3D000F1189644271773004E73004FDC504353C7
:10F3E000C30001DD50DC4EC9008900DD4E397F00CD
:10F3F0004E7F004F9649D6553DDD50D655272F9666
:10F4000048270B3DD34FDD4F964E8900974ED6557A
:10F410009647270A3DD34EDD4E24037EF4ACD655E5
:10F420009646270A3D4D26F3DB4E25EFD74ED654A0
:10F4300027389649270B3DD34FDD4F964E890097CD
:10F440004ED654964827083D4DD34E25CEDD4EF678
:10F45000C420C1452614D6549647270A3D4D26BBE5
:10F46000DB4E25B7D74E964626B1D653272396496D
:10F4700027093DD34EDD4E2533974ED65396482768
:10F480000A3D4D2627DB4E2523D74E96479A462622
:10F490001BD65227169649270A3D4D260FDB4E25CF
:10F4A0000BD74E96489A479A46260139CC00077EDC
:10F4B000F118BDF01125433736863DBDEFF4263AED
:10F4C000BDE4FEDF46380FDC52ED00DC54ED020EE9
:10F4D000DF52DE4639863ABDEFF4260532327ECB66
:10F4E00023860DBDEFF426063232087ECAED39BD03
:10F4F000F004810D27F8813A27F43C4F5FCEF12DBF
:10F500000EDD547F00527F0053CCFB1DDDAC7F002D
:10F51000B57D008127273CFE71788CFFFF38271DC1
:10F5200096B681182606BDFB1D7F00B68E7FFFCCE8
:10F530000000FD717AFD7180DE82BDCAFB7F00B3E1
:10F540007F00B496B6270CBDFB1D96B68118260326
:10F550007F00B64FBDF696860AB776E0DC542709E1
:10F560007F0045BDF6D1BDF815FE71788CFFFF26F2
:10F57000037ECE03EC0026037EC71CBDF76B183854
:10F5800009DF4618A600810D270FBDF8179C4626F7
:10F5900005863FBDF8170820EBBDF8177EC71C3C59
:10F5A000CEF1334F5F7EF500C60DD74636DF5218D9
:10F5B000C300F0DD54DE52BDFAE0817F27418108AF
:10F5C000273D810A27F1810027ED8103261133377A
:10F5D000C13A260B33383838FF7178387EF838A7AF
:10F5E00000089146261233C13A270CBDFB1D810D40
:10F5F0002605860ABDFB1D39BDFB1D9C5426B89C03
:10F600005227B4098608BDFB1D8620BDFB1D860858
:10F61000BDFB1D20A2DE548C80002508CC00087E96
:10F62000F1183232DEB1BC718E25040D86FF39EC43
:10F6300000847F9354250139E602DF564FD35618D4
:10F6400020E4200108A6002AFB20DB3CDE5227072D
:10F6500038CC00087EF118DE548C800024F2FE7154
:10F6600078EC00847F26035D27B8189C543825D297
:10F67000FE7178200C09E6000886FF50DF56D3564D
:10F6800018DC548A80A1002605E1012601399CB1CD
:10F6900026E30D86FF3916A60008112601393637F4
:10F6A000BDF8173332810D26EE398622BDEFF426E0
:10F6B0000ABDF696810D2601094F398627BDEFF464
:10F6C00027EF817F260A81082606860D9DAB20E95B
:10F6D000393C964536848097449645847F97458685
:10F6E00014367A0045F676E0C10A260E7D00522ACD
:10F6F00009BDF17F7C00447A0045F676E04F18DFC3
:10F70000487F00477F0046BDF2BADE522604DE5431
:10F710002708D651377A004520E0D651377B804400
:10F720002715964484012704862D9DAB7A00452B2E
:10F730001B86309DAB20F57A00452B0686209DABBD
:10F7400020F5964484012704862D9DAB3281142731
:10F750000C810A25028B078B309DAB20EF32974539
:10F760003839BDF76B4FBDF6960839EC00847FDD64
:10F77000547F00527F005308080886049745BDF661
:10F78000D18620BDF81739FE7190BC7194260139DD
:10F79000A600083CFE7192A70008FF71923820EA8B
:10F7A000FE7196BC719A26013909A6003CFE71983B
:10F7B00009A700FF71983820EA3233DF5E38FF7105
:10F7C00080271838FF718638FF718838FF718238BA
:10F7D000FF718438FF718A38FF718C3736DE5E39ED
:10F7E0003233DF5E308C77132405DE5E7EF59FFEBC
:10F7F0007180271BFE718C3CFE718A3CFE71843C3B
:10F80000FE71823CFE71883CFE71863CFE71803C3C
:10F810003736DE5E39860D369DAB3236810D2604D5
:10F82000860A9DAB32397D00932601397D009E27E3
:10F83000FA7F0093BDFA7E0E7D008C271A8E7FFD25
:10F84000CC0000FD717AFD7180CC0064DD54CC00E9
:10F8500000DD523C7ECB32FE71782727CEF886BD84
:10F86000F8154FBDF696FE7178EC00847FDD547F6D
:10F8700000527F00537F0045860AB776E0BDF6D17F
:10F88000BDF8157EC71C425245414B204154204CC7
:10F89000494E45200039BDF895BDF8BE7B02BB2717
:10F8A000193C18C601BDE07672101771EF1772107F
:10F8B0001771EF17724017183839724017390F3C1B
:10F8C0001896171684CF971784BF9717188604C108
:10F8D000082505722017200371DF1772101771EFCA
:10F8E0001758C40F4A26E8961716CA10D717971745
:10F8F000D7179717D7179717D7179717D717971798
:10F90000D7179D28CE000409010101010126F8CE78
:10F91000000A4F5F057B08172702CB407210177152
:10F92000EF170926EF724017380E399752D7467FE6
:10F9300000530F3C71DF1771BF17CE000A7210170A
:10F9400071EF170926F7CE00030901010101012615
:10F95000F87C005396539754CE000A4F5F71EF170F
:10F960007800547B10542705722017200371DF178D
:10F97000057B081727015C7210170926E0369617D9
:10F9800084EF9D28320E38050505050505BDF9A053
:10F990009652915327043C7EF9467240177EF8BA7E
:10F9A0007D004627167A004626057C004620087C06
:10F9B000004637BDF1E232BDF1E23905057B02BBFD
:10F9C00027F5050520F1961E84D02755845027037E
:10F9D00096123BDE719612A7007B017627128113E7
:10F9E0002605728076203A81112605717F762031B6
:10F9F000810326037C0093098C70732603CE7173F8
:10FA0000DF717D0075261A189373C1402613FC76AA
:10FA1000DCB376DAC1FF27098613BDFB1D86FF978D
:10FA20007596118424812427013B7B017627237B53
:10FA30008076271EDEAFBDF82671FB110E01019600
:10FA4000431A914327F90F0927057B807626E77132
:10FA50007F76FE76DCA600098C75D92603CE76D992
:10FA6000FF76DC7D007726029713FE76DCBC76DA23
:10FA7000260471FB113B7204113B86FF97753CCE47
:10FA80007173DF71DF7371FB11CE76D9FF76DAFF08
:10FA900076DC967527088611BDFB1D7F00753871D1
:10FAA0007F767F0093399674907239B676DDB076A2
:10FAB000DB39DE643CDE663CDEB3EC00DD64EC0288
:10FAC000DD663CBDF22138D664E700D665E701D695
:10FAD00066E702D667E70338DF6638DF6433383914
:10FAE0003C3736DCB33226CADE739C7126031A20FB
:10FAF000F7A60036098C70732603CE7173DF7396F8
:10FB000075270F189371C14026088611BDFB1D7F14
:10FB10000075323338810326037A0093393C373637
:10FB2000FC76DCB376DAC1FF27F6FE76DA32A70080
:10FB3000098C75D92603CE76D9FF76DA7204113393
:10FB4000383986209DAB86209DAB393B3B86059797
:10FB5000908E00FF9614C6FFD7053686E097148670
:10FB600012971BB6C41F8B0C971C7F00017F0020CF
:10FB70007F008B7F008A860A971186059710C6F052
:10FB800086F07F00BBD71797169770867EB7010F58
:10FB9000CCFC36FD0110865F7B01BB270286BF9738
:10FBA0001C9763860197B897B772401B0ECE000072
:10FBB000DF42DF407F00AE32848027068E7FFF7EEB
:10FBC000C6A6CE7FFDCE0000DF9ADF9C5FCEFC068E
:10FBD0003AA600CE75BD3AA7005CC11826EF5FCEED
:10FBE000FC1E3AA600CE00283AA7005CC11826EFFA
:10FBF000867E97949797CCF258DD95CCF255DD9898
:10FC00008E7FFF7EC6AC717F17F78000A7007280E1
:10FC10001739717F17F78000A60072801739DE2828
:10FC2000DE28DE28010101010101010101010101BC
:10FC3000010101971739DE6C08DF6C7A00B82619CC
:10FC4000DC42C30001DD42DC40C9008900DD409692
:10FC5000AE890097AE96B797B8717F1B3B2A2020DC
:10FC600050433D2420413D2420423D2420463D2454
:10FC700020583D242040583D242053503D2420400E
:10FC800024DEAC3CCEFB1DDFAC0E860DBDFB1D861D
:10FC90000ABDFB1DCEFC5DBDFD193C30EC09180909
:10FCA000BDFD2138BDFD193C30A606BDFD2638BD81
:10FCB000FD193C30A605BDFD2638BDFD193C30A61A
:10FCC00004BDFD2638BDFD193C30EC0718BDFD21F3
:10FCD00038BDFD193C30EC0718EC0018BDFD21388B
:10FCE000BDFD193C3018C3000A18BDFD2138BDFD0B
:10FCF00019FE706ABDFD21863DBDFB1DFE706A8642
:10FD00000836A60008BDFD268620BDFB1D324A260A
:10FD1000F038DFAC3BBDFB1D08A600812426F608A9
:10FD2000393C328D013236444444448D0132840FD3
:0BFD30008B30813A25028B077EFB1D03
:10FFC7007EFAAB7EF8BE7EF8957EF89C7EF1A47E25
:10FFD700F1B87EFAA67EFAE07EFB1D7EFA7E7EF8F9
:10FFE7009600DF0100010FFB4BF9C6010301060173
:09FFF70009010CFC81FB4CFB4DDF
:00000001FF
